:0200000480007A
:10000000B72F0000938F0F8073900F3015A8130047
:100010000000130000001300000013000000130094
:100020000000130000001300000013000000130084
:100030000000130000001300000013000000010086
:10004000970200009382020C73905230814001416C
:100050008141014281420143814301448144014580
:100060008145014681460147814701488148014950
:100070008149014A814A014B814B014C814C014D20
:10008000814D014E814E014F814F971102009381A6
:1000900021C1170502001305E542979503009385DA
:1000A000657501461122170502001305A53E970547
:1000B00002009385A53E0146C52817A50300130538
:1000C000A57397B503009385E57237B6ABAB1306FE
:1000D000B6BAD92817B1030013010172EF40F0013D
:1000E000860293D21200F512638802008242110147
:1000F0006F00001073002030824211017300203025
:10010000711116C0F3222034E3CC02FC82421101AB
:10011000130141F806C20AC40EC612C816CA1ACC88
:100120001ECE22D026D22AD42ED632D836DA3ADCC7
:100130003EDEC2C0C6C2CAC4CEC6D2C8D6CADACC97
:10014000DECEE2D0E6D2EAD4EED6F2D8F6DAFADCA7
:10015000FEDE73252034F32510340A8601A07310C7
:10016000153492402241B2414242D2426243F243AC
:10017000025492542255B2554256D2566257F25703
:10018000064896482649B649464AD64A664BF64B33
:10019000065C965C265DB65D465ED65E665FF65F83
:1001A0001301C1077300203010C16374B50011053D
:1001B000E5BF828000000000000000000000000099
:1001C000000000000000000000000000000000002F
:1001D000000000000000000000000000000000001F
:1001E000000000000000000000000000000000000F
:1001F000197106C00AC20EC412C616C81ACA1ECC8D
:1002000022CE26D02AD22ED432D636D83ADA3EDCC6
:1002100042DEC6C0CAC2CEC4D2C6D6C8DACADECC96
:10022000E2CEE6D0EAD2EED4F2D6F6D8FADAFEDCA6
:100230009702020083A2022623A02200F322103498
:1002400096DEEF006030170102000321A124024175
:10025000F65273901234B72200009382028873A082
:10026000023082403242C2425243E24372448254DC
:100270001255A2553256C2565257E2577258864806
:100280001649A649364AC64A564BE64B764C865C1A
:10029000165DA65D365EC65E565FE65F0961730059
:1002A0002030970202009382E22123A0120023A2B1
:1002B000220023A4320023A6420023A8520023AA2E
:1002C000620023AC720023AE820023A0920223A21C
:1002D000A20223A4B20223A6C20223A8D20223AA06
:1002E000E20223ACF20223AE020323A0120523A2F2
:1002F000220523A4320523A6420523A8520523AADA
:10030000620523AC720523AE820523A0920723A2C7
:10031000A20723A4B20723A6C20723A8D20723AAB1
:10032000E20723ACF207EF40804D170102000321E2
:1003300061160241F65273901234B7220000938284
:10034000028873A0023082403242C2425243E243EA
:10035000724482541255A2553256C2565257E25731
:10036000725886481649A649364AC64A564BE64B45
:10037000764C865C165DA65D365EC65E565FE65FB1
:10038000096173002030970202009382A21383A0B8
:10039000020003A1420083A1820003A2C20083A243
:1003A000020103A3420183A3820103A4C20183A427
:1003B000020203A5420283A5820203A6C20283A60B
:1003C000020303A7420383A7820303A8C20383A8EF
:1003D000020403A9420483A9820403AAC20483AAD3
:1003E000020503AB420583AB820503ACC20583ACB7
:1003F000020603AD420683AD820603AEC20683AE9B
:10040000020703AFC20983AF820782807370043092
:10041000197106C00AC20EC412C616C81ACA1ECC6A
:1004200022CE26D02AD22ED432D636D83ADA3EDCA4
:1004300042DEC6C0CAC2CEC4D2C6D6C8DACADECC74
:10044000E2CEE6D0EAD2EED4F2D6F6D8FADAFEDC84
:100450009702020083A2020423A0220086DEEF108E
:10046000B040170102000321E1020241F6527390ED
:100470001234B72200009382028873A002308240B7
:100480003242C2425243E243724482541255A25550
:100490003256C2565257E257725886481649A649F4
:1004A000364AC64A564BE64B764C865C165DA65DD0
:1004B000365EC65E565FE65F0961730020309707BF
:1004C00002009387E7FD9843FD576305F7007370BB
:1004D000043001A07370043001A041112AC6B24754
:1004E000739047300100410182804111F327403071
:1004F0003EC673F04330B2473E85410182804111D0
:100500002AC62EC432C2B247F1173EC62247B247AE
:1005100098C3B247938787FA3EC61247B24798C33B
:10052000B247A1173EC68E873E87B24798C3B247EF
:10053000D1173EC6170700001307A7F8B24798C3A4
:10054000B2473E8541018280411106C6EF40A0239B
:10055000EF10D014AA8799C3EF1010310100B240F8
:100560004101828041112AC6B24713878700B247F2
:10057000D8C3B2477D5798C7B24713878700B247A1
:10058000D8C7B24713878700B24798CBB24723A09A
:10059000070001004101828041112AC6B24723A809
:1005A000070001004101828001112AC62EC4B24712
:1005B000DC433ECEA2477247D8C3F2479847A247D2
:1005C00098C7F2479C472247D8C3F247224798C7AB
:1005D000A247324798CBB2479C4313871700B247D4
:1005E00098C301000561828001112AC62EC4A2476A
:1005F0009C433ECC6247FD576316F700B2479C4BC5
:100600003ECE31A8B247A1073ECE21A0F247DC433F
:100610003ECEF247DC439C436247E379F7FEF24764
:10062000D843A247D8C3A247DC43224798C7A24772
:10063000724798C7F2472247D8C3A247324798CBA0
:10064000B2479C4313871700B24798C30100056166
:10065000828001112AC6B2479C4B3ECEB247DC4392
:100660003247184798C7B2479C4732475843D8C3C8
:10067000F247DC4332476316F700B2479847F24728
:10068000D8C3B24723A80700F2479C431387F7FF5C
:10069000F24798C3F2479C433E8505618280797199
:1006A00006D622D42AC62EC4B2473ECEF24781E7F0
:1006B0007370043001A0EF202057F2478043F247C7
:1006C000D85FF247BC43BE853A85EF50F043AA8716
:1006D0003307F400F247D8C3F24723AC0702F247CE
:1006E0009843F24798C7F2478043F247DC5F13878D
:1006F000F7FFF247BC43BE853A85EF50F040AA872A
:100700003307F400F247D8C7F2477D57F8C3F247E2
:100710007D57B8C7A24799EFF2479C4B8DC7F24768
:10072000C1073E85EF1090402A878547631DF7007B
:10073000F13911A8F247C1073E852D35F24793875D
:1007400047023E850535EF20005185473E85B25072
:10075000225445618280797106D62AC62EC4B2879A
:10076000A303F10002CCB24781E77370043001A00B
:10077000A24799E302CE01A8A2453245EF50D038F6
:10078000AA8785073ECEF247938747053E85EF301F
:10079000805C2ACAD24785CFA24789E7D247524711
:1007A00098C331A0D24713874705D24798C3D24791
:1007B0003247D8DFD2472247B8C385455245C535B1
:1007C000D247034771002388E704D2473ECCE24773
:1007D00081E77370043001A0E2473E85B250456165
:1007E0008280797106D6AA87A307F1001305400518
:1007F000EF3060562ACEF247B9CFF24723A2070066
:10080000F24723A00700F24723A40700F24723A6DC
:100810000700F24723AC0702F2470547D8DFF2474B
:1008200023A00704F2477D57F8C3F2477D57B8C7A6
:10083000F2470347F1002388E704F247C1073E85EA
:100840001533F247938747023E85293B814601468F
:10085000814572453122F2473E85B2504561828022
:10086000797106D622D42AC6B2473ECCE24781E748
:100870007370043001A0E247C043EF20001DAA8737
:100880006313F402E247DC471387F7FFE247D8C758
:10089000E247DC4791E78146014681456245C92030
:1008A00085473ECE11A002CEF2473E85B25022547B
:1008B00045618280797106D622D42AC62EC4B247F9
:1008C0003ECCE24781E77370043001A0E247C043A9
:1008D000EF20A017AA87631BF400E247DC471387C9
:1008E0001700E247D8C785473ECE0DA08146224675
:1008F00081456245252E2ACE724785476318F70049
:10090000E247DC4713871700E247D8C7F2473E8526
:10091000B250225445618280797106D62AC62EC40F
:10092000B24781E77370043001A02247B24763F5F4
:10093000E7007370043001A0094681453245213D2E
:100940002ACEF24781C7F247224798DFF24781E774
:100950007370043001A0F2473E85B2504561828039
:10096000397106DE2AC62EC432C236C002D6B2475C
:100970003ED4A25781E77370043001A0A24781E7FB
:10098000A257BC4399E3854711A0814781E7737063
:10099000043001A0024789476317F700A257D85FC8
:1009A00085476314F700854711A0814781E773707D
:1009B000043001A0EF20C00AAA8799E3924799E387
:1009C000854711A0814781E77370043001A0EF20B3
:1009D000A025A257985FA257DC5F6366F700024725
:1009E0008947631DF7020246A245225565232AD294
:1009F000A257DC5389CFA257938747023E85EF1059
:100A0000F0122A8785476317F700093421A092570F
:100A100091C3ED3AEF202024854771A8924789E7DA
:100A2000EF206023814741A8B25799E77C083E85B3
:100A3000EF10702785473ED6EF20E021EF10401AD7
:100A4000EF20801EA257F843FD576315F700A25709
:100A500023A20704A257B847FD576315F700A25712
:100A600023A40704EF20201F58007C08BA853E8588
:100A7000EF107026AA879DEB2255EF006071AA87C0
:100A80008DC3A257C1071247BA853E85EF10E070AB
:100A900022551525EF108016AA87E39A07F2BD327A
:100AA0003DB72255092DEF10601515B722552125A8
:100AB000EF10C01481473E85F25021618280797128
:100AC00006D62AC62EC432C236C0B2473ECCE24752
:100AD00081E77370043001A0A24781E7E247BC437D
:100AE00099E3854711A0814781E77370043001A025
:100AF000024789476317F700E247D85F85476314C9
:100B0000F700854711A0814781E77370043001A089
:100B1000E93AAA873ECAE247985FE247DC5F63662C
:100B2000F700024789476315F7040246A24562456C
:100B30009521E247B847FD576313F702E247DC53BC
:100B40008DC7E247938747023E85EF10207EAA8734
:100B500089CF924799CB9247054798C339A0E2477E
:100B6000BC4713871700E247B8C785473ECE11A0A0
:100B700002CED2473E859532F2473E85B25045615E
:100B80008280797106D62AC62EC4B2473ECCE2478F
:100B900081E77370043001A0E247BC4381C77370E2
:100BA000043001A0E2479C4381E7E247DC4399E33C
:100BB000854711A0814781E77370043001A0353269
:100BC000AA873ECAE247985FE247DC5F6377F70493
:100BD000E2479C5F13871700E24798DFE247B84778
:100BE000FD576313F702E247DC538DC7E247938753
:100BF00047023E85EF108073AA8789CFA24799CB21
:100C0000A247054798C339A0E247BC47138717009E
:100C1000E247B8C785473ECE11A002CED2473E85F7
:100C20006D38F2473E85B25045618280397106DEEB
:100C30002AC62EC432C236C002D6B2473ED4A2570C
:100C400081E77370043001A0A24781E7A257BC433B
:100C500099E3854711A0814781E77370043001A0B3
:100C6000EF101060AA8799E3924799E3854711A096
:100C7000814781E77370043001A0EF10F07AA2572A
:100C80009C5FB5CBA257DC473ED2A2452255F92E38
:100C9000824795EFA2579C5F1387F7FFA25798DF13
:100CA000A2579C4391E7EF2060022A87A257D8C33E
:100CB000A2579C4B8DCFA257C1073E85EF1000670E
:100CC0002A8785476315F702EFF04FF40DA0A2576E
:100CD0001257D8C7A257DC5399CBA2579387470224
:100CE0003E85EF10A064AA8799C3EFF02FF2EF10B2
:100CF000907685475DA8924789E7EF10D0758147C8
:100D00006DA0B25799E77C083E85EF10C079854702
:100D10003ED6EF105074EF00B06CEF10F070A25799
:100D2000F843FD576315F700A25723A20704A25703
:100D3000B847FD576315F700A25723A40704EF1027
:100D4000907158007C08BA853E85EF10C078AA875C
:100D5000A1EB2255CD2EAA879DCFA2579C4391EBA4
:100D6000EF10906CA257DC433E85EF107052EF10ED
:100D7000906EA257938747021247BA853E85EF10BF
:100D8000C04122550D2EEF007067AA87E39707EE4A
:100D9000EFF0CFE7DDB52255392EEF003066F1BD1B
:100DA0002255112EEF00906581473E85F25021615A
:100DB0008280797106D62AC62EC432C2B2473ECC92
:100DC000E24781E77370043001A0A24781E7E24760
:100DD000BC4399E3854711A0814781E773700430D4
:100DE00001A0EFF08FF0AA873ECAE2479C5FA1CB3B
:100DF000A2456245A52CE2479C5F1387F7FFE247B7
:100E000098DFE247F843FD576312F702E2479C4B35
:100E100085C7E247C1073E85EF104051AA8789CFB9
:100E2000924799CB9247054798C339A0E247FC43C4
:100E300013871700E247F8C385473ECE11A002CEC4
:100E4000D2473E85EFF06FE9F2473E85B2504561EB
:100E50008280797106D62AC62EC4B2473ECCE247BC
:100E600081E77370043001A0A24781E7E247BC43E9
:100E700099E3854711A0814781E77370043001A091
:100E8000E247BC4381E77370043001A0EFF0EFE567
:100E9000AA873ECAE2479C5F89CFE247DC473EC84B
:100EA000A2456245E122E2474247D8C785473ECE88
:100EB00011A002CED2473E85EFF02FE2F2473E85E9
:100EC000B25045618280797106D62AC6B24781E761
:100ED0007370043001A0EF103055B2479C5F3ECED6
:100EE000EF107057F2473E85B250456182807971AC
:100EF00006D62AC6B2473ECEF24781E77370043069
:100F000001A0EF107052F247D85FF2479C5FB30721
:100F1000F7403ECCEF103054E2473E85B250456179
:100F2000828001112AC6B24781E77370043001A0A4
:100F3000B2479C5F3ECEF2473E8505618280797163
:100F400006D62AC6B2473ECEF24781E77370043018
:100F500001A07245E5247245EF20F0720100B25005
:100F60004561828041112AC6B247FC473E85410156
:100F7000828041112AC62EC4B2472247F8C7010019
:100F80004101828041112AC6B24783C707053E85C9
:100F900041018280797106D62AC62EC432C202CEA1
:100FA000B247BC4391EFB2479C43D5E7B247DC431D
:100FB0003E85EF10903B2ACEB24723A2070061A8DE
:100FC000924785EFB2479847B247BC433E86A24559
:100FD0003A85EF20F079B2479847B247BC433E9735
:100FE000B24798C7B2479847B247DC436365F706F4
:100FF000B2479843B24798C7B9A8B247D847B24753
:10100000BC433E86A2453A85EF209076B247D8474A
:10101000B247BC43B307F0403E97B247D8C7B24788
:10102000D847B2479C43637BF700B247D843B247E7
:10103000BC43B307F0403E97B247D8C71247894731
:10104000631BF700B2479C5F99C7B2479C5F138749
:10105000F7FFB24798DFB2479C5F13871700B2478C
:1010600098DFF2473E85B25045618280011106CE7D
:101070002AC62EC4B247BC439DCBB247D847B2471D
:10108000BC433E97B247D8C7B247D847B247DC43C4
:101090006366F700B2479843B247D8C7B247D8470C
:1010A000B247BC433E86BA852245EF20706C0100F2
:1010B000F24005618280011106CE2AC6EF10D036BB
:1010C00025A0B247DC5395C7B247938747023E85B8
:1010D000EF10C025AA8799C3EF104049B247BC471B
:1010E0001387F7FFB247B8C7B247BC47E34BF0FCE2
:1010F00011A00100B2477D57B8C7EF10D035EF10EF
:10110000B0321DA0B2479C4B8DC7B247C1073E8588
:10111000EF10C021AA8799C3EF104045B247FC43A6
:101120001387F7FFB247F8C3B247FC43E34CF0FC28
:1011300011A00100B2477D57F8C3EF10D031010074
:10114000F24005618280797106D62AC6EF10D02D53
:10115000B2479C5F81E785473ECE11A002CEEF10DB
:10116000902FF2473E85B2504561828001112AC618
:10117000B24781E77370043001A0B2479C5F81E7FA
:1011800085473ECE11A002CEF2473E8505618280A2
:10119000797106D62AC6EF103029B247985FB24758
:1011A000DC5F6315F70085473ECE11A002CEEF103D
:1011B000902AF2473E85B2504561828001112AC6CD
:1011C000B24781E77370043001A0B247985FB2471D
:1011D000DC5F6315F70085473ECE11A002CEF247D3
:1011E0003E850561828001112AC62EC402CE81A0EF
:1011F000178703001307475CF2478E07BA979C4393
:1012000085E7178703001307275BF2478E07BA9716
:10121000224798C3178703001307075AF2478E0720
:10122000BA973247D8C301A8F24785073ECE724726
:101230009D47E3FFE7FA01000561828001112AC69C
:1012400002CE0DA81787030013070757F2478E0732
:10125000BA97DC433247631CF70017870300130774
:10126000A755F2478E07BA9723A0070001A8F247B7
:1012700085073ECE72479D47E3F6E7FC0100056116
:101280008280797106D62AC62EC432C2B2473ECEBB
:10129000EF109019F247F843FD576315F700F24736
:1012A00023A20704F247B847FD576315F700F2473A
:1012B00023A40704EF10301AF2479C5F89EBF24732
:1012C000938747021246A2453E85EF00907E724505
:1012D000DD330100B25045618280397106DE2ACECD
:1012E0002ECC36C83AC63EC442C246C0B287231B83
:1012F000F100F24781E77370043001A03247914753
:1013000063F5E7007370043001A0835761019245D3
:101310003E85EF1080512AD4A257638F0712A2573F
:10132000985B83566101B7070040FD17B6978A079F
:10133000BA973ED29257F19B3ED292578D8B81C77E
:101340007370043001A0835761013E8782463246A4
:10135000E2452255EF10E0274246F2451255EFF0E4
:101360000F9A2A87A25798C3A24781C7A24722573C
:1013700098C3EF10700B97F701009387A7299C4340
:101380001387170097F701009387C72898C397F72B
:101390000100938727109C4395E397F701009387FB
:1013A000670F225798C397F701009387A7269843A2
:1013B0008547631AF702EF10C02C35A097F701009C
:1013C000938707269C4385E397F701009387870C53
:1013D0009C43DC5732476368F70097F70100938717
:1013E000670B225798C397F70100938767249C43A4
:1013F0001387170097F701009387872398C397F700
:1014000001009387E7229843A257B8C7A257D8573D
:1014100097F70100938787209C4363F9E700A25761
:10142000D85797F701009387671F98C3A257D857DB
:10143000BA878A07BA978A0717F701001307471078
:101440003E97A2579107BE853A85EFF0EF95854705
:101450003ED6EF10500019A0FD573ED632578547B3
:101460006313F70297F701009387871B9C4381CF93
:1014700097F70100938707029C43DC57324763F4D8
:10148000E700EFE0BFF8B2573E85F250216182805D
:10149000797106D62AC6EF102079B24799E797F7F7
:1014A0000100938727FF9C4311A0B2473ECEF2472D
:1014B00091073E85EFF0EF99F2479C5791C7F247AD
:1014C000E1073E85EFF0EF98F2479107BE8517F5EB
:1014D000010013056511EFF02F8D97F70100938739
:1014E000E7119C431387170097F7010093870711B3
:1014F00098C397F701009387A7139C43138717009E
:1015000097F701009387C71298C3EF10C07497F73D
:1015100001009387E7109C439DCB97F701009387C9
:1015200067F79C437247631EF70097F701009387A4
:10153000A7109C4381C77370043001A0EFE01FED3A
:1015400039A0EF10606EEF10A04BEF10C0700100DB
:10155000B25045618280797106D62AC62EC402CE69
:10156000B24781E77370043001A0A24781E773702E
:10157000043001A097F701009387070C9C4381C7B3
:101580007370043001A0A92D97F701009387C70855
:101590009C433ECCB2479C432247BA973ECAB247CF
:1015A0009C436247637EF700B2479C435247637493
:1015B000F7025247E24763F0E70285473ECE21A893
:1015C000B2479C4352476366F7005247E24763F4D1
:1015D000E70085473ECEB247524798C3F24789CFCE
:1015E00097F70100938707EB9C4391073E85EFF047
:1015F0004F865245EF10001B11252AC8C24799E3B8
:10160000EFE0DFE00100B25045618280797106D6DB
:101610002AC602CEB247A9C397F701009387C70134
:101620009C4381C77370043001A05D2B97F70100C4
:10163000938787FE9C433247BA973ECC97F70100C9
:10164000938747E59C4391073E85EFF08F80624585
:10165000EF10401565232ACEF24799E3EFE01FDB38
:101660000100B25045618280797106D62AC6B24720
:101670003ECCE24781E77370043001A097F7010088
:10168000938747E19C4362476314F70002CEBDA0F5
:10169000EF108059E247DC4B3ECAEF10C05B97F772
:1016A00001009387A7F29C435247630AF70097F71C
:1016B00001009387E7F19C4352476315F700894780
:1016C0003ECE2DA8524797F70100938767F3631B1F
:1016D000F700E2479C5781E78D473ECE05A089473A
:1016E0003ECE29A8524797F701009387E7EF63158D
:1016F000F70091473ECE19A085473ECEF2473E8582
:10170000B25045618280797106D62AC6EF10C05169
:10171000B24799E797F701009387C7D79C4311A079
:10172000B2473ECEF247DC573ECCEF10C052E24704
:101730003E85B25045618280797106D62AC6EFE0B7
:10174000DFDAAA873ECEB24799E797F70100938781
:1017500067D49C4311A0B2473ECCE247DC573ECA57
:10176000F2473E85EFE07FD7D2473E85B2504561D4
:101770008280797106D62AC62EC402CE22479147AE
:1017800063F5E7007370043001A02247914763F4CA
:10179000E70091473EC4EF102049B24799E797F719
:1017A0000100938727CF9C4311A0B2473ECCE2476C
:1017B000BC4B3ECA5247A247630AF70E2247D247A4
:1017C00063F6E70297F701009387C7CC9C43624713
:1017D0006308F70297F701009387C7CB9C43DC5758
:1017E0002247636FF70085473ECE19A897F701009F
:1017F000938747CA9C4362476314F70085473ECEF0
:10180000E247DC573EC8E247B84BE247DC57631576
:10181000F700E2472247D8D7E2472247B8CBE24752
:101820009C4F63C707001547A2471D8FE24798CF1B
:10183000E247D44B4247BA878A07BA978A0717F715
:1018400001001307E7CFBA976394F600854711A00C
:101850008147B9C7E24791073E85EFE09FDFE24746
:10186000D85797F70100938767DB9C4363F9E7003C
:10187000E247D85797F70100938747DA98C3E247C2
:10188000D857BA878A07BA978A0717F7010013074C
:1018900027CB3E97E2479107BE853A85EFE0DFD040
:1018A000724785476314F700EFE05FB6EF10A03A88
:1018B0000100B25045618280797106D62AC6EF10C8
:1018C000A036B24799E797F701009387A7BC9C43DE
:1018D00011A0B2473ECEF24791073E85EFE07FD799
:1018E000F2479C5791C7F247E1073E85EFE07FD66C
:1018F000F2479107BE8517F50100130565D0EFE0AB
:10190000BFCAEF10403597F701009387A7B89C43F3
:1019100072476319F70497F70100938767D09C43D8
:1019200089CF97F70100938727D19C4381C77370B4
:10193000043001A0EFE09FAD91A097F701009387DD
:1019400027CC984397F701009387C7CC9C43631932
:10195000F70097F701009387E7B323A0070039A8A2
:10196000212729A897F70100938787CB9C4399C724
:10197000EF10802BEF10C008EF10E02D0100B250E7
:101980004561828001112AC602CEB2473ECCB247E1
:1019900081E77370043001A0E247D84B97F701004C
:1019A000938707C66314F700854711A0814795C345
:1019B000E247985797F701009387C7C1630BF70079
:1019C000E2479C5799E3854711A0814799C3854712
:1019D0003ECEF2473E8505618280797106D62AC6E1
:1019E000B2473ECEB24781E77370043001A0F247A0
:1019F000C9C797F701009387E7A99C437247630E15
:101A0000F706EF1060227245B53F2A8785476314B9
:101A1000F706F24791073E85EFE0BFC3F247D8577C
:101A200097F70100938787BF9C4363F9E700F2476C
:101A3000D85797F70100938767BE98C3F247D857E6
:101A4000BA878A07BA978A0717F70100130747AFC3
:101A50003E97F2479107BE853A85EFE0FFB4F24723
:101A6000D85797F701009387E7A29C43DC5763643C
:101A7000F700EFE0BF99EF10001E0100B250456182
:101A80008280797106D62AC602CEB2473ECCB247D2
:101A900081E77370043001A0EFE03FA5AA873ECA3A
:101AA0006245CD352A8785476314F70897F701000B
:101AB000938787B89C43A5E7E247D85797F701007B
:101AC0009387479D9C43DC576364F70085473ECE70
:101AD000E24791073E85EFE0DFB7E247D85797F737
:101AE00001009387A7B39C4363F9E700E247D85707
:101AF00097F70100938787B298C3E247D857BA8710
:101B00008A07BA978A0717F70100130767A33E975A
:101B1000E2479107BE853A85EFE01FA911A8E24789
:101B2000E107BE8517F501001305C5AAEFE0DFA7A1
:101B3000D2473E85EFE07F9AF2473E85B25045613D
:101B40008280011106CE81480148814701478146C4
:101B50001306004097E501009385C54A171500005C
:101B6000130585A5EFF06FF72AC632478547631541
:101B7000F700EF10C06D2AC6324785476319F70298
:101B80007370043097F701009387C7AA7D5798C3F5
:101B900097F701009387C7A8054798C397F70100F7
:101BA000938787A723A00700EFE0AFEF31A0B247EC
:101BB00081E77370043001A00100F240056182806A
:101BC000411106C67370043097F70100938747A54B
:101BD00023A00700EFE02FFB0100B240410182800B
:101BE00097F70100938747A59C431387170097F742
:101BF0000100938767A498C301008280011106CE7B
:101C000002C697F70100938727A39C4381E773706F
:101C1000043001A0EF10400197F701009387C7A19E
:101C20009C431387F7FF97F701009387E7A098C3BA
:101C300097F70100938747A09C436390071097F79D
:101C400001009387279D9C436389070E59A097F74E
:101C5000010093872798DC47DC473EC4A247E10791
:101C60003E85EFE01F9FA24791073E85EFE07F9EF4
:101C7000A247D85797F701009387479A9C4363F987
:101C8000E700A247D85797F701009387279998C391
:101C9000A247D857BA878A07BA978A0717F7010069
:101CA0001307078A3E97A2479107BE853A85EFE062
:101CB000BF8FA247D85797E701009387A77D9C4322
:101CC000DC576368F70097F701009387E7950547AE
:101CD00098C397F701009387E78F9C43ADFB97F775
:101CE0000100938727949C438DCF35A0452AAA876E
:101CF00099C797F7010093872793054798C397F7EC
:101D00000100938727929C431387F7FF97F7010001
:101D10009387479198C397F701009387A7909C43B7
:101D2000F1F797F70100938727909843854763164B
:101D3000F70085473EC6EFE06FEDEF00D071B24788
:101D40003E85F24005618280011106CEEF00D06D24
:101D500097F701009387478C9C433EC6EF00B06F16
:101D6000B2473E85F24005618280011106CEEFE068
:101D7000CFF7AA873EC697F701009387E7899C4370
:101D80003EC4B2473E85EFE04FF5A2473E85F240A4
:101D90000561828097F701009387C7879C433E8542
:101DA0008280797106D62AC62EC432C202CE9547E9
:101DB0003ECC3D3597F701009387C7859C4322476A
:101DC0006368F70CE247FD173ECCF24796073247AF
:101DD000B306F7006247BA878A07BA978A0717E7F8
:101DE00001001307E775BA970546BE853685EF00F3
:101DF000902A2A87F247BA973ECEE247E1F7F247A8
:101E0000960732473E9797E701009387277C9C43CC
:101E10000946BE853A85EF0010282A87F247BA970F
:101E20003ECEF247960732473E9797E701009387E9
:101E3000277A9C430946BE853A85EF00D0252A873C
:101E4000F247BA973ECEF24796073247BA97114605
:101E500097E50100938545793E85EF00D0232A87D9
:101E6000F247BA973ECEF24796073247BA970D46E9
:101E700097E501009385C5783E85EF00D0212A873C
:101E8000F247BA973ECE924781C7924723A00700F8
:101E9000B533F2473E85B25045618280797106D6EE
:101EA00002CE97E70100938727799C436395071833
:101EB00097E70100938747769C431387170097E7BE
:101EC00001009387677598C397E701009387C774EC
:101ED0009C433ECCE247B9EF97E701009387076F39
:101EE0009C439C4381C77370043001A097E70100B5
:101EF0009387C76D9C433ECA97E701009387476D60
:101F0000984397E701009387676C98C397E70100B0
:101F10009387076C524798C397E70100938707712F
:101F20009C431387170097E701009387277098C396
:101F3000EF00102D97E701009387C76F9C4362471E
:101F40006365F70C97E70100938747689C439C43C0
:101F500099E3854711A0814781CB97E701009387DB
:101F6000676D7D5798C355A097E701009387076673
:101F70009C43DC47DC473EC8C247DC433EC6624761
:101F8000B2476379F70097E701009387A76A324762
:101F900098C3A5A8C24791073E85EFE08FEBC247E3
:101FA0009C5791C7C247E1073E85EFE08FEAC247E1
:101FB000D85797E70100938767669C4363F9E7006A
:101FC000C247D85797E701009387476598C3C24730
:101FD000D857BA878A07BA978A0717E70100130705
:101FE00027563E97C2479107BE853A85EFE0CFDB83
:101FF000C247D85797E701009387C7499C43DC57EE
:10200000E362F7F485473ECE35BF97E7010093873B
:1020100067489C43D85797E6010093866652BA8773
:102020008A07BA978A07B6979843854763F1E7020C
:1020300085473ECE29A897E701009387A75E9C437A
:102040001387170097E701009387C75D98C397E749
:1020500001009387675D9C4399C385473ECEF24755
:102060003E85B25045618280011106CE97E701009E
:102070009387875C9C4381CB97E701009387C75A7E
:10208000054798C339A297E701009387E75923A032
:10209000070097E701009387E73F9C439C5B3EC6A0
:1020A000B7A7A5A59387575A3EC4B2479C4322477A
:1020B0006314F702B24791079C432247631EF7005F
:1020C000B247A1079C4322476318F700B247B10704
:1020D0009C4322476308F70497E701009387873BF7
:1020E000984397E701009387E73A9C439387470318
:1020F000BE853A85EF20B00F35A097E701009387A2
:10210000E7519C4381E77370043001A097E7010019
:102110009387C7509C431387F7FF97E70100938786
:10212000E74F98C397E701009387474F984397E697
:1021300001009386E640BA878A07BA978A07B6975E
:102140009C43C5DF97E701009387474D9843BA87C3
:102150008A07BA978A0717E701001307673EBA97FD
:102160003EC29247DC43D8439247D8C39247D843F4
:102170009247A1076317F7009247DC43D843924781
:10218000D8C39247DC43D84797E70100938787304D
:1021900098C30100F24005618280797106D62AC693
:1021A0002EC4B24781E77370043001A097E70100A5
:1021B0009387472E9C43E107BE853245EFE0CFC2AF
:1021C00097E701009387072D9C4391073E85EFE039
:1021D0004FC82247FD576310F70297E70100938726
:1021E000672B9C439107BE8517E501001305454108
:1021F000EFE08FBB19A897E701009387E7419C4365
:102200002247BA973ECE7245712B0100B25045610C
:102210008280797106D62AC62EC432C2B24781E7BF
:102220007370043001A097E701009387E7409C4357
:1022300081E77370043001A097E701009387872539
:102240009C43A24637070080558F98CF97E701003F
:10225000938747249C43E107BE853245EFE0CFB426
:1022600097E70100938707239C4391073E85EFE0A2
:102270004FBE1247FD576310F70297E7010093879F
:1022800067219C439107BE8517E50100130545377B
:10229000EFE08FB119A897E701009387E7379C43D8
:1022A0001247BA973ECE7245F5290100B2504561FA
:1022B0008280797106D62AC62EC432C2B24781E71F
:1022C0007370043001A097E701009387A71C9C431B
:1022D000E107BE853245EFE02FAD97E70100938718
:1022E000671B9C4391073E85EFE0AFB612478547D9
:1022F0006310F70297E701009387C7199C43910782
:10230000BE8517E501001305A52FEFE0EFA919A879
:1023100097E70100938747309C432247BA973ECE08
:10232000724549210100B25045618280797106D61B
:102330002AC6B247DC47DC473ECCE24781E77370F0
:10234000043001A0E247E1073E85EFE08FB097E758
:1023500001009387672E9C43A1EBE24791073E85DE
:10236000EFE02FAFE247D85797E701009387072B9D
:102370009C4363F9E700E247D85797E7010093874A
:10238000E72998C3E247D857BA878A07BA978A07D6
:1023900017E701001307C71A3E97E2479107BE856A
:1023A0003A85EFE06FA011A8E247E107BE8517E587
:1023B000010013052522EFE02F9FE247D85797E74A
:1023C00001009387270D9C43DC5763FBE70085479B
:1023D0003ECE97E7010093872725054798C311A0B4
:1023E00002CEF2473E85B25045618280797106D6B1
:1023F0002AC62EC497E70100938707249C4381E7F0
:102400007370043001A02247B70700805D8FB24788
:1024100098C3B247DC473ECCE24781E77370043093
:1024200001A03245EFE0EFA2E24791073E85EFE0E1
:102430004FA2E247D85797E701009387271E9C4396
:1024400063F9E700E247D85797E701009387071D34
:1024500098C3E247D857BA878A07BA978A0717E717
:1024600001001307E70D3E97E2479107BE853A85C5
:10247000EFE08F93E247D85797E7010093878701F2
:102480009C43DC5763FBE70085473ECE97E701009E
:1024900093878719054798C311A002CEF2473E855E
:1024A000B2504561828041112AC6B24781E77370FC
:1024B000043001A097E70100938747179843B2477C
:1024C00098C397E70100938727159843B247D8C36D
:1024D000010041018280797106D62AC62EC4B24716
:1024E00081E77370043001A0A24781E77370043064
:1024F00001A01D2F97E70100938707129C433ECC54
:10250000A2479843FD576314F70002CE91A8B24743
:10251000984397E70100938767119C43630AF7008C
:10252000B247DC4362476365F70085473ECE0DA89E
:10253000B247DC4362471D8FA2479C436370F7029A
:10254000A2479843B247D443E247B387F6403E9749
:10255000A24798C33245813F02CE19A085473ECE9F
:10256000DD2DF2473E85B2504561828097E701003C
:102570009387870B054798C30100828001112AC603
:10258000B24799C7B2473ECCE247FC473ECE11A0C6
:1025900002CEF2473E850561828001112AC62EC413
:1025A000B24791C7B2473ECEF2472247F8C7010073
:1025B00005618280011106CE2AC6852297E70100B7
:1025C000938707F898438547E3F9E7FEEFD01FE4C8
:1025D000EDB7397106DE2ACE2ECC32CA36C8BA879C
:1025E0002317F10002D625A06247B257BA9703C756
:1025F0000700F246B257B697238AE7026247B257FE
:10260000BA9783C7070089CBB25785073ED63257A2
:10261000BD47E3FBE7FC11A00100F247A3810704DB
:102620005247914763F4E70091473ECAF247524749
:10263000D8D7F2475247B8CBF24723AA0704F2474C
:1026400091073E85EFD05FF5F247E1073E85EFD079
:10265000BFF4F247724798CB1547D2471D8FF24718
:1026600098CFF2477247D8D3F24723A20704F24724
:1026700023AC0704F24723AE07040100F2502161A6
:102680008280011106CE02C60DA03247BA878A07A2
:10269000BA978A0717E70100130787EABA973E85BA
:1026A000EFD05FECB24785073EC632479147E3FE65
:1026B000E7FC17E501001305E5EEEFD0BFEA17E5EB
:1026C0000100130565EFEFD0FFE917E501001305E1
:1026D00065F0EFD03FE917E501001305E5F0EFD015
:1026E0007FE817E501001305A5F1EFD0BFE797E7F5
:1026F00001009387A7ED17E701001307A7EA98C326
:1027000097E701009387C7EC17E701001307C7EAB3
:1027100098C30100F24005618280011106CE8DA8A8
:10272000EFF00FCC97E70100938707EC9C4393B73A
:10273000170093F7F70F3EC6EFF04FCCB247A9EB67
:10274000E52197E70100938727EADC47DC473EC491
:10275000A24791073E85EFD0DFEF97E7010093870F
:1027600067EB9C431387F7FF97E70100938787EA9E
:1027700098C397E70100938767E89C431387F7FFA7
:1027800097E70100938787E798C3F1212245912CB1
:1027900097E70100938787E69C43D9F30100F24055
:1027A00005618280011106CE2AC697E70100938752
:1027B00067CE9C433247D8C397E701009387C7E5AC
:1027C0009C4332476372F70297E70100938747E023
:1027D000984397E701009387E7CB9C439107BE8519
:1027E0003A85EFD07FE035A897E70100938707DEB1
:1027F000984397E701009387E7C99C439107BE85FB
:102800003A85EFD07FDE97E701009387A7E29C43EC
:1028100032476378F70097E701009387A7E13247D3
:1028200098C30100F24005618280797106D6AA87BB
:102830002EC42317F100A24789EB8357E1008A07D2
:102840003E85EF104051AA8711A0A2473ECCE24737
:1028500085C313050006EF1000502ACEF24789C742
:10286000F247624798DB31A06245EF10C06111A0CA
:1028700002CEF24781CFF247985B8357E1008A0787
:102880003E869305500A3A85EF104075F2473E8523
:10289000B25045618280397106DE22DC2AC62EC420
:1028A00032C202D6A2479C43638D070EA2473ED494
:1028B000A257DC43D843A257D8C3A257D843A25744
:1028C000A1076317F700A257DC43D843A257D8C328
:1028D000A257DC43DC473ED2A2473ED08257DC43BE
:1028E000D8438257D8C38257D8438257A10763176A
:1028F000F7008257DC43D8438257D8C38257DC4362
:10290000DC473ECEB25796073247BA97724798C314
:10291000B25796073247BA97724713074703D8C38F
:10292000B25796073247BA977247384798C7B25797
:1029300096073247BA971247D8C7B2579607324719
:10294000BA977247585798CB12478D47631BF700C9
:10295000F2479C5799C7B25796073247BA9709472B
:10296000D8C7B25796073247BA977247384BD8CB79
:10297000B25796073247BA9723AC0700F247945BE9
:10298000B257960732473304F70036850D20AA87E1
:10299000231EF400B25785073ED672479257E31DB7
:1029A000F7F2B2573E85F2506254216182800111E4
:1029B0002AC602CE39A0B24785073EC6F247850730
:1029C0003ECEB24703C707009307500AE305F7FE60
:1029D000F24789833ECEF247C207C1833E85056137
:1029E0008280011106CE2AC6B2479C5B3E85EF105D
:1029F00080493245EF1020490100F2400561828094
:102A0000411197E70100938767BC9C439C4399E37E
:102A1000854711A0814781CB97E70100938787C144
:102A20007D5798C305A097E70100938727BA9C4379
:102A3000DC47DC473EC6B247D84397E7010093879F
:102A400067BF98C3010041018280411197E70100EF
:102A5000938747A49C433EC6B2473E85410182808E
:102A6000411197E701009387A7BB9C4381E7854706
:102A70003EC619A897E70100938707BC9C4381E7EE
:102A800089473EC611A002C6B2473E8541018280F9
:102A9000797106D62AC6B2473ECEB247F9C3F2478D
:102AA000D85797E701009387E79E9C43DC57637AEA
:102AB000F70AF2479C4F63CC070097E70100938722
:102AC000679D9C43DC5715471D8FF24798CFF2470F
:102AD000D44BF247D857BA878A07BA978A0717E7BD
:102AE00001001307E7A5BA976394F600854711A084
:102AF0008147A5C3F24791073E85EFD09FB597E781
:102B00000100938727999C43D857F247D8D7F247BB
:102B1000D85797E70100938767B09C4363F9E700B4
:102B2000F247D85797E70100938747AF98C3F2471A
:102B3000D857BA878A07BA978A0717E70100130799
:102B400027A03E97F2479107BE853A85EFD0DFA5D3
:102B500009A897E701009387E7939C43D857F2476A
:102B6000D8D70100B25045618280797106D62AC655
:102B7000B2473ECC02CEB247DDC397E70100938750
:102B800067919C4362476305F7007370043001A0AE
:102B9000E247FC4B81E77370043001A0E247FC4B35
:102BA0001387F7FFE247F8CBE247D857E247BC4B21
:102BB0006307F706E247FC4BBDE3E24791073E851A
:102BC000EFD03FA9E247B84BE247D8D7E247DC57FE
:102BD00015471D8FE24798CFE247D85797E7010086
:102BE0009387C7A39C4363F9E700E247D85797E769
:102BF00001009387A7A298C3E247D857BA878A07EC
:102C0000BA978A0717E70100130787933E97E247B1
:102C10009107BE853A85EFD03F9985473ECEF24772
:102C20003E85B250456182807370043097E70100A1
:102C30009387079F9C4391CF97E7010093878785F0
:102C40009C43F8430507F8C397E7010093878784FF
:102C50009C430100828097E701009387679C9C4317
:102C60008DCB97E701009387E7829C43FC4395C394
:102C700097E70100938707829C43F8437D17F8C3C9
:102C800097E70100938707819C43FC4399E37360B6
:102C9000043001008280411197D701009387877F1C
:102CA0009C439C4F3EC697D701009387A77E9C43C9
:102CB000D85797D701009387E77D9C439546338784
:102CC000E64098CFB2473E854101828097D7010008
:102CD0009387477C9C4389CB97D701009387877B59
:102CE0009C43F84B0507F8CB97D701009387877A69
:102CF0009C433E858280797106D62AC62EC42D3724
:102D000097D70100938707799C43BC4FADE397D7D2
:102D10000100938727789C430547F8CFA247A1CBB2
:102D200097D70100938707779C4391073E85EFD0A3
:102D30005F922247FD576310F70297D701009387F0
:102D400067759C439107BE8517E501001305458B08
:102D5000EFD09F8519A897E701009387E78B9C43E5
:102D60002247BA973ECE7245353CEFD02FEAE53583
:102D7000653D97D701009387E7719C43BC4F3ECCDC
:102D8000E2479DC3B24789CB97D7010093878770ED
:102D90009C4323AC070409A897D701009387876F4A
:102DA0009C43B84F7D17B8CF97D701009387876EA4
:102DB0009C4323AE07044535E2473E85B25045614A
:102DC0008280797106D62AC62EC432C236C0A93D89
:102DD00097D701009387076C9C43F84F8947630D91
:102DE000F70697D701009387E76A9C43B44F3247B1
:102DF0001347F7FF758FB8CF97D70100938787697F
:102E00009C430547F8CF8247A1CB97D70100938712
:102E100067689C4391073E85EFD0BF830247FD570B
:102E20006310F70297D701009387C7669C43910709
:102E3000BE8517D501001305A57CEFD0EFF619A8C4
:102E400097D701009387477D9C430247BA973ECCB2
:102E50006245893AEFD08FDBFD3BF933924789CB4E
:102E600097D70100938707639C43B84F924798C355
:102E700097D70100938707629C43F84F85476314F7
:102E8000F70002CE31A897D701009387A7609C4333
:102E9000B44F22471347F7FF758FB8CF85473ECE13
:102EA00097D701009387075F9C4323AE07046533E0
:102EB000F2473E85B25045618280797106D62AC6B6
:102EC0002EC432C236C085473ECEB24781E773700A
:102ED000043001A0B2473ECC813B824789C7E2471C
:102EE000B84F824798C3E247FC4F3ECAE2470947C2
:102EF000F8CF1247914763EEE704924713972700F4
:102F000097D7010093878710BA97984397D7010006
:102F10009387C70FBA978287E247B84FA2475D8F62
:102F2000E247B8CF3DA0E247BC4F13871700E24706
:102F3000B8CF05A0E2472247B8CF21A8524789471A
:102F40006306F700E2472247B8CF21A002CE11A0C6
:102F5000010052478547631AF706E24791073E850D
:102F6000EFD02FEFE247D85797D701009387076B31
:102F70009C4363F9E700E247D85797D7010093874E
:102F8000E76998C3E247D857BA878A07BA978A078A
:102F900017D701001307C75A3E97E2479107BE852E
:102FA0003A85EFD06FE0E2479C5781C773700430D9
:102FB00001A0E247D85797D701009387A74D9C43BC
:102FC000DC5763F4E700EFD06FC47131F2473E8500
:102FD000B25045618280397106DE2ACE2ECC32CACB
:102FE00036C83AC685473ED6F24781E7737004304B
:102FF00001A0F2473ED4EFD04FCFAA873ED2C247BE
:1030000089C7A257B84FC24798C3A257FC4F3ED0BA
:10301000A2570947F8CF5247914763EEE704D247DA
:103020001397270097D70100938787FFBA97984394
:1030300097D701009387C7FEBA978287A257B84FE8
:10304000E2475D8FA257B8CF3DA0A257BC4F138770
:103050001700A257B8CF05A0A2576247B8CF21A842
:10306000025789476306F700A2576247B8CF21A0ED
:1030700002D611A0010002578547631DF708A25729
:103080009C5781C77370043001A097D701009387C4
:10309000A75A9C43A1EBA25791073E85EFD06FDB67
:1030A000A257D85797D70100938747579C4363F996
:1030B000E700A257D85797D701009387275698C3A0
:1030C000A257D857BA878A07BA978A0717D7010035
:1030D000130707473E97A2579107BE853A85EFD061
:1030E000AFCC11A8A257E107BE8517D50100130583
:1030F000654EEFD06FCBA257D85797D70100938773
:1031000067399C43DC5763F7E700B24781C7B24792
:10311000054798C392573E85EFD02FBCB2573E85E6
:10312000F25021618280797106D62AC62EC4B24738
:1031300081E77370043001A0B2473ECEEFD0EFBA02
:10314000AA873ECCF247FC4F3ECAF2470947F8CF68
:10315000F247BC4F13871700F247B8CF5247854755
:10316000631DF708F2479C5781C77370043001A0B4
:1031700097D701009387474C9C43A1EBF2479107F7
:103180003E85EFD00FCDF247D85797D701009387F0
:10319000E7489C4363F9E700F247D85797D7010007
:1031A0009387C74798C3F247D857BA878A07BA9711
:1031B0008A0717D701001307A7383E97F2479107F0
:1031C000BE853A85EFD04FBE11A8F247E107BE8514
:1031D00017D5010013050540EFD00FBDF247D857B2
:1031E00097D701009387072B9C43DC5763F7E700D1
:1031F000A24781C7A247054798C3E2473E85EFD063
:10320000CFAD0100B25045618280797106D62AC6E1
:10321000B2473ECCE24799E797D7010093878727CB
:103220009C4311A0E2473ECC0134E247F84F894766
:103230006318F700E24723AE070485473ECE11A08E
:1032400002CE113CF2473E85B250456182800111A9
:1032500006CE02C61D2B97D70100938727419C43BA
:103260009DC38148014881470947814613060040B4
:1032700097D50100938505DC170500001305051B94
:10328000EFE0AF852AC6B24781E77370043001A032
:10329000B2473E85F24005618280397106DE2ACE52
:1032A0002ECC32CA36C83AC6E24799E302D62DA8D8
:1032B0001305C002EF00302A2AD6B25795C7F12174
:1032C000B257724798C3B257624798CFB257524726
:1032D000D8CFB257424798D3B2573247D8D3B25714
:1032E00091073E85EFD04FABE24781E77370043022
:1032F00001A0B2573E85F25021618280397106DE0D
:103300002ACE2ECC32CA36C83AC602D6F24781E758
:103310007370043001A097D70100938727359C4331
:10332000B5CBE2473ED0D2473ED2F2473ED46247C9
:10333000954763C4E704EFF0AFF22A87894763102B
:10334000F70297D70100938767329C431810814694
:103350003246BA853E85EFD0AFE02AD625A897D76A
:1033600001009387A7309C43181081460146BA8517
:103370003E85EFD0EFDE2AD631A897D7010093879C
:10338000E72E9C43181081464246BA853E85EFD011
:103390000FF32AD6B2573E85F25021618280011187
:1033A0002AC6B2473ECEB24781E77370043001A00F
:1033B000F2479C433E8505618280797106D62AC614
:1033C0002EC497D701009387E7299C43DC47DC474D
:1033D0003ECEF24791073E85EFD0AFA7F247D84FD8
:1033E0008547631BF702F247984FB247BA97B24638
:1033F0002246BE857245B9222A878547631EF7009B
:1034000001478146324681457245CD3D2ACCE2478F
:1034100081E77370043001A0F247DC537245829754
:103420000100B25045618280797106D62AC63C08F7
:103430003E8541282ACEE247BE8572451920692281
:10344000FDB7797106D62AC62EC4EFE06FF93C08A5
:103450003E8545282ACEE247B9EFA24799EB32478D
:10346000F24763E8E700EFE06FF9F2453245B13724
:10347000A9A0A24781CF97D701009387E71E9C435D
:103480009C4393B7170093F7F70F3EC497D70100FB
:103490009387C71D94433247F247B307F74022464C
:1034A000BE853685EFD0FFDDEFE04FF5AA8791E7C7
:1034B000EFC0DFF519A0EFE06FF40100B2504561F5
:1034C000828001112AC697D701009387A7199C43D0
:1034D0009C4393B7170093F7F70F3E87B24798C303
:1034E000B2479C4391EB97D701009387A7179C4362
:1034F000DC479C433ECE11A002CEF2473E850561DB
:103500008280797106D62AC6EFE01F842ACE97D72B
:1035100001009387E7159C4372476377F700692A98
:10352000B247054798C321A0B24723A0070097D709
:1035300001009387E713724798C3F2473E85B25064
:1035400045618280797106D62AC62EC432C236C041
:1035500002CEB2472247D8C3B247324798CB224760
:10356000924763E8E702124782471D8FB2479C4F9C
:103570006365F70085473ECE99A097D701009387F2
:10358000A70E9843B2479107BE853A85EFD0CF8505
:103590003DA0124782476379F7002247824763655F
:1035A000F70085473ECE21A897D701009387870B68
:1035B0009843B2479107BE853A85EFD0EF82F24734
:1035C0003E85B25045618280797106D6D9A0A24766
:1035D00063C0070CC2473ECEF247DC4B91C7F247AF
:1035E00091073E85EFD0EF865C003E85193F2ACCDF
:1035F000A2472547636FF7081397270097D7010065
:103600009387C7A3BA97984397D70100938707A3D7
:10361000BA9782873247F2479C4FBA973247BA86A9
:103620006246BE857245393F2A8785476313F70690
:10363000F247DC5372458297F247D84F8547631AA9
:10364000F7043247F2479C4FBA97014781463E86BE
:103650008145724565312ACAD24785EF73700430BF
:1036600001A03247F24798CFF2479C4F81E7737031
:10367000043001A0F247984FE247BA97E24662460B
:10368000BE857245C13531A07245EF00C07F11A0E3
:10369000010097D70100938767FD9C43380081465E
:1036A0000146BA853E85EFD06FD8AA87E39107F22D
:1036B0000100B25045618280797106D671A097D71A
:1036C0000100938727FA9C43DC479C433ECC97D765
:1036D0000100938727F99C43DC47DC473ECAD24769
:1036E00091073E85EFC0FFF6D247DC5352458297E3
:1036F000D247D84F85476319F704D2479C4F62479A
:10370000BA973EC84247E24763F4E702D2474247CE
:10371000D8C3D247524798CB97D70100938787F4F5
:103720009843D2479107BE853A85EFC0FFEB29A8A1
:1037300001478146624681455245C9362AC6B2478D
:1037400081E77370043001A097D70100938787F158
:103750009C439C43ADF797D701009387A7F09C4308
:103760003ECE97D70100938727F0984397D7010063
:10377000938747EF98C397D701009387E7EE724787
:1037800098C30100B25045618280411106C6EFF036
:10379000AFC997D70100938767ED9C43C9E717D559
:1037A00001001305A5E9EFC0FFDB17D501001305E4
:1037B00025EAEFC03FDB97D701009387A7EA17D729
:1037C00001001307A7E798C397D701009387C7E9BC
:1037D00017D701001307C7E798C30146B145114544
:1037E000EFC07FF72A8797D70100938727E898C310
:1037F00097D70100938787E79C4381E77370043074
:1038000001A097D70100938767E69C4389CF97D79C
:1038100001009387A7E59C4397D501009385858494
:103820003E85EFD05F9CEFF00FC30100B240410135
:103830008280797106D62AC6B2473ECEB24781E76A
:103840007370043001A0EFF02FBEF247DC4BB337AA
:10385000F00093F7F70F3ECCEFF0EFBFE2473E8565
:10386000B25045618280797106D62AC6B2473ECEF3
:10387000B24781E77370043001A0EFF0EFBAF2476E
:103880009C533ECCEFF02FBDE2473E85B2504561E0
:103890008280797106D62AC62EC4B2473ECEB24780
:1038A00081E77370043001A0EFF00FB8F2472247B0
:1038B00098D3EFF04FBA0100B250456182800111F8
:1038C00006CE714549292AC6B24789CBB24723A003
:1038D0000700B24791073E85EFC0DFC8B2473E857B
:1038E000F24005618280397106DE2AC62EC432C2DA
:1038F00036C0B2473ED402D21247B70700FFF98F55
:1039000081C77370043001A0924781E7737004305F
:1039100001A0EFF0EF94AA8799E3824799E38547E6
:1039200011A0814781E77370043001A0EFE04FAB35
:10393000A2579C433ED0A245324585240257A24758
:103940005D8F9247F98F12476310F7020257A24723
:10395000D98F3ED6A2579843924793C7F7FF7D8FE2
:10396000A25798C302C025A0824799CFA257938639
:1039700047001247B7070005D98F0246BE85368536
:10398000EFE03F8902D621A0A2579C433ED6EFE04C
:10399000EFA62ACE8247B1CBF24799E3EFC01FA72B
:1039A000EFF06FAF2AD63257B7070002F98F85EBD9
:1039B000EFF08FA7A2579C433ED632579247F98F1C
:1039C0001247631AF700A2579843924793C7F7FF2D
:1039D0007D8FA25798C3EFF00FA885473ED232578C
:1039E000B7070001FD17F98F3ED6B2573E85F2505A
:1039F000216182805D7186C62ACE2ECC32CA36C83D
:103A00003AC6F2473EDA02DC02D8F24781E7737029
:103A1000043001A06247B70700FFF98F81C77370B8
:103A2000043001A0E24781E77370043001A0EFF099
:103A30002F83AA8799E3B24799E3854711A081476D
:103A400081E77370043001A0EFE08F99D2579C4357
:103A50003ED64246E245325575242AD4A25799CF24
:103A6000B2573EDE02C6D247A9CBD2579843E247AF
:103A700093C7F7FF7D8FD25798C381A0B24781E7E4
:103A8000B2573EDE1DA8D24791C76257B707000163
:103A9000D98F3EDCC24791C76257B7070004D98F60
:103AA0003EDCD257938647006247E257D98F3246B1
:103AB000BE853685EFE0EFF502DEEFE02F942AD2E7
:103AC000B247B9CB925799E3EFC05F94EFF0AF9C48
:103AD0002ADE7257B7070002F98F8DEBEFF0CF9413
:103AE000D2579C433EDE4246E2457255212CAA87BE
:103AF00099CBD24789CBD2579843E24793C7F7FF78
:103B00007D8FD25798C3EFF00F9502D87257B70741
:103B10000001FD17F98F3EDEF2573E85B640616128
:103B20008280797106D62AC62EC4B2473ECEB247ED
:103B300081E77370043001A02247B70700FFF98FB7
:103B400081C77370043001A0EFF00F8EF2479C43E1
:103B50003ECCF2479843A24793C7F7FF7D8FF247C9
:103B600098C3EFF04F8FE2473E85B25045618280A7
:103B7000797106D62AC6B2473ECEEFC01F97AA87F4
:103B80003ECCF2479C433ECAE2473E85EFC0FF94DD
:103B9000D2473E85B250456182805D7186C62AC695
:103BA0002EC402DCB2473ED802DAB24781E7737016
:103BB000043001A02247B70700FFF98F81C7737057
:103BC000043001A0C25791073ED6B257A1073ED498
:103BD000EFE00F81B257DC473EDEC2579843A24761
:103BE0005D8FC25798C3BDA8F257DC433ED2F2574F
:103BF0009C433ED002DA0257B70700FFF98F3ECE52
:103C00000257B7070001FD17F98F3ED07247B7077B
:103C10000004F98F89EBC25798438257F98F89CFF7
:103C200085473EDA11A8C25798438257F98F025749
:103C30006314F70085473EDAD2579DC37247B70732
:103C40000001F98F89C762578257D98F3EDCC2576E
:103C50009843B7070002D98FBE857255EFE00FF980
:103C600092573EDE7257A257E310F7F8C2579843B7
:103C7000E25793C7F7FF7D8FC25798C3EFD01FF865
:103C8000C2579C433E85B64061618280797106D6F9
:103C90002AC6B2473ECEF24791073ECCEFD05FF442
:103CA0000DA0E247D847E247A1076315F7007370FC
:103CB000043001A0E247DC47B70500023E85EFE093
:103CC000EFF2E2479C43F1FF7245752AEFD01FF3F4
:103CD0000100B25045618280011106CE2AC62EC471
:103CE000A24532455D3D0100F2400561828001112F
:103CF00006CE2AC62EC4A245324525350100F24023
:103D00000561828001112AC62EC432C202CE9247BA
:103D100081EB3247A247F98F81CF85473ECE09A874
:103D20003247A247F98F22476314F70085473ECEFA
:103D3000F2473E850561828001112AC6B2473ECC1A
:103D4000B24799E302CE21A0E2479C4F3ECEF24714
:103D50003E8505618280397106DE2AC602D2EFD027
:103D60003FE8976703009387E7919C4381EB5522D7
:103D70009767030093870791054798C3B24789CF98
:103D8000A1473E87B247BA973EC6B2478D8B89C7D7
:103D9000B247F19B91073EC6B247F9CB3247E56780
:103DA000ED1763E7E70C976703009387A78C3ED472
:103DB000976703009387078C9C433ED631A0B25788
:103DC0003ED4B2579C433ED6B257DC43324763F5EC
:103DD000E700B2579C43E5F7325797670300938794
:103DE000E7896307F708A2579C432147BA973ED259
:103DF000B2579843A25798C3B257D843B247B307B4
:103E0000F740214706076378F7043257B247BA975D
:103E10003ECEB257D843B2471D8FF247D8C3B257F0
:103E20003247D8C3F247DC433ECC97670300938701
:103E300067843ED021A082579C433ED082579C434A
:103E4000DC436247E3E9E7FE82579843F24798C3B1
:103E50008257724798C397C701009387E7649843D6
:103E6000B257DC431D8F97C701009387E76398C360
:103E7000EFD0DFD8925799E3EF00D03692573E85C6
:103E8000F25021618280797106D62AC6B2473ECCB3
:103E9000B247BDC3A147B307F0406247BA973ECCD3
:103EA000E2473ECAEFD0DFD3D247DC433EC8975744
:103EB00003009387277C3ECE21A0F2479C433ECE51
:103EC000F2479C43DC434247E3E9E7FEF24798436D
:103ED000D24798C3F247524798C3D247D84397C7AF
:103EE00001009387675C9C433E9797C701009387C7
:103EF000A75B98C3EFD09FD00100B250456182808C
:103F000097C701009387475A9C433E8582800100F2
:103F10008280411197C7010093870776F19B3EC6C7
:103F20009757030093870775324798C39757030045
:103F30009387477423A2070097570300938707745A
:103F400065677117D8C3975703009387277323A01A
:103F50000700B2473EC4A24765677117D8C3A2479E
:103F6000175703001307877198C30100410182802E
:103F700001112AC62EC432C2A2473ECEB2473ECC61
:103F80003247A247D98F8D8BA1E319A8F2479843F6
:103F9000E24798C3E24791073ECCF24791073ECEF5
:103FA0009247F5173247BA976247E361F7FE29A8AF
:103FB0007247930717003ECEE2479386170036CC30
:103FC000034707002380E70032479247BA976247CA
:103FD000E360F7FEB2473E850561828001112AC683
:103FE0002EC432C232479247D98F8D8B9DEFA247A4
:103FF00093F7F70F3ECAD247A2075247D98F3ECA5E
:10400000D247C2075247D98F3ECAB2473ECE39A0E7
:10401000F247138747003ACE524798C33247924738
:10402000BA977247E366F7FE1DA0B2473ECC11A8CF
:10403000E247138717003ACC22471377F70F238004
:10404000E70032479247BA976247E363F7FEB24709
:104050003E850561828001112AC6B2473ECE21A06D
:10406000F24785073ECEF24783C70700F5FB72474C
:10407000B247B307F7403E850561828001112AC629
:104080002EC4B247138717003AC683C70700A30F91
:10409000F100A247138717003AC483C70700230F14
:1040A000F1008347F10199C70347F1018347E1011B
:1040B000E309F7FC0347F1018347E101B307F74048
:1040C0003E850561828001112AC62EC4B2473ECECC
:1040D00001002247930717003EC4F247938617005A
:1040E00036CE034707002380E70083C70700F5F3B8
:1040F000B2473E850561828001112AC602CE02CCFC
:1041000021A0B24785073EC6B24703C70700930701
:104110000002E308F7FEB24703C707009307D00287
:104120006309F700B24703C707009307B0026311A2
:10413000F704B24783C70700938737FD93B717008B
:1041400093F7F70F3ECCB24785073EC615A07247DE
:10415000BA878A07BA9786073ECEB24713871700F9
:104160003AC683C70700938707FD7247BA973ECECA
:10417000B24783C70700E1FFE24789C7F247B307A9
:10418000F04011A0F2473E850561828001112AC6E8
:1041900097570300938707539C439386170017573D
:1041A00003001307275214C332471377F70F9756AC
:1041B000030093862655B6972380E7003247A94728
:1041C000630BF700975703009387C74F98439307F4
:1041D00000046315F704975703009387A7523ECE58
:1041E00005A8F247138717003ACE03C70700B707A1
:1041F00010F0938707F098C3975703009387874C75
:104200009C431387F7FF975703009387A74B98C3E7
:10421000975703009387074B9C43E1F781473E85FF
:10422000056182804D7123261114232481142322D9
:10423000911423202115232E3113232C4113232ADB
:1042400051132ACE2ECC32C836CA3AC63EC442C218
:1042500023260112B2473E8A814AC24752485286FB
:10426000D6863E85C285EF10303AAA872E883E86D4
:10427000C2868327C112138717002326E1123287D3
:104280008A07141AB69723AEE7EEB2473E848144FC
:10429000D247268763E8E702D24726876396E7007E
:1042A000C247228763E0E702B2473E8981494A86D6
:1042B000CE864245D245EF106057AA872E883EC869
:1042C00042CA49BF010029A0F247E2451245829740
:1042D000A2471387F7FF3AC40327C112E346F7FE4C
:1042E00025A88327C1128A07181ABA9703A7C7EF10
:1042F0008327C1128A07141AB69783A6C7EFA5476A
:1043000063F5D7009307700519A093070003BA97C8
:104310007247E2453E8502978327C1121387F7FF54
:104320002326E112E34FF0FA01008320C114032495
:10433000811483244114032901148329C113032AFE
:104340008113832A41137161828041112AC62EC4D0
:10435000A2460547635ED700B2479C439D07E19B99
:1043600093868700324714C303A847009C4335A0B7
:10437000224719CB3247184313064700B24690C272
:104380001843BA87014811A832471843130647005B
:10439000B24690C21843BA8701483E85C2854101A2
:1043A000828041112AC62EC4A2460547635ED7000B
:1043B000B2479C439D07E19B93868700324714C315
:1043C00003A847009C4305A8224701CF3247184362
:1043D00013064700B24690C21843BA877D873A88D1
:1043E00019A83247184313064700B24690C2184333
:1043F000BA877D873A883E85C285410182803971BE
:1044000006DE22DC26DA2AC62EC432C236C011A845
:1044100063070424924785073EC2B247A24522851E
:104420008297924783C707003E8493075002E311A7
:10443000F4FE924785073EC292473EC893070002AA
:10444000A30BF100FD573ECEFD573ECC02D0924764
:10445000138717003AC283C707003E849307D4FD31
:10446000130750056364F71E1397270097C70100D1
:10447000938747C0BA97984397C70100938787BF30
:10448000BA9782879307D002A30BF100C9B79307AD
:104490000003A30BF10065BF02CC6247BA878A070D
:1044A000BA978607A297938707FD3ECC924783C7AA
:1044B00007003E849307F00263D6870293079003B8
:1044C00063C28702924785073EC2C1BF82471387F6
:1044D00047003AC09C433ECC39A0F247E3D907F6E7
:1044E00002CEB5B70100F247E3D307F6E2473ECE6E
:1044F000FD573ECCA9BF825785073ED089BF824772
:10450000138747003AC09C433247A2453E85029735
:10451000B1A28247138747003AC0844389E497C415
:1045200001009384A4B4F2476357F0040347710178
:104530009307D0026301F704E247BE852685EF109A
:10454000A02C2A87F247998F3ECE11A8834771018C
:104550003247A2453E850297F247FD173ECEF2470D
:10456000E346F0FE09A8B247A2452285829785045A
:10457000F247FD173ECE83C704003E841DC0E247CC
:10458000E3C307FEE247FD173ECCE247E3DD07FC4D
:1045900009A8B247A245130500028297F247FD170A
:1045A0003ECEF247E347F0FE55A88A8782553E8506
:1045B000CD3BAA872E883ED442D6A2573258C28716
:1045C00063D90702B247A2451305D0028297A255CC
:1045D000325681470148B386B740368533B5A700C8
:1045E0003307C840B307A7403E87B6873A883ED412
:1045F00042D6A9473ED21DA8A9473ED215A0A14741
:104600003ED239A885473ED0B247A24513050003E4
:104610008297B247A245130580078297C1473ED2D1
:104620008A8782553E8515332AD42ED61257834762
:1046300071013E88F2472256B256A2453245DD3618
:1046400031A8B247A2452285829709A8B247A24560
:10465000130550028297C2473EC20100D9B3010040
:10466000F2506254D2542161828041112AC6B707A8
:1046700010F0938707F2324798C301A05D7106D608
:104680002AC62EDA32DC36DEBAC0BEC2C2C4C6C604
:104690009C0891173ECEF247BE86324681451705EB
:1046A00000001305E5AEA13B81473E85B250616134
:1046B000828001112AC62EC41EC2A2473ECEF247F6
:1046C0009C4332471377F70F2380E700F2479C4360
:1046D00013871700F24798C30100056182801D719E
:1046E00006DE2AC62EC4B2C4B6C6BAC8BECAC2CC7A
:1046F000C6CE9C103ED25C084C081706000013067C
:1047000086FB7D779346F7FF0565130505803388A3
:10471000A5003378E8001368783B23A007013295A1
:10472000698F13677733D8C333F7D50093154701E3
:1047300037870300130737394D8F98C73377D60073
:10474000931647013707030013077706558FD8C71D
:104750000F100000B2473ED69C10A1173ED422573E
:104760005C083E857C00BA862246BE854939B24740
:1047700023800700B2473E87B257B307F7403E8514
:10478000F250256182804111370510F0130545F480
:1047900008412AC6370510F0130505F408412AC45C
:1047A000370510F0130545F40841B248E39EA8FC14
:1047B00032452A8381431317030081462245AA8587
:1047C0000146B3E7B6003368C700370710F013059A
:1047D00087F48565938585380146B386B700B6882A
:1047E000B3B8F8003307C800B387E8003E87B68740
:1047F0003A881CC123220501010041018280411138
:1048000006C651379307000873A047300100B24035
:1048100041018280011106CE2AC617C50100130589
:10482000E59AEFF0BFE50100F240056182800111D9
:1048300006CE2AC617C501001305C599EFF01FE47F
:104840000100F24005618280797106D62AC602CE47
:1048500029A00100F24785073ECE724785679387FE
:104860007738E3D8E7FE17C5010013052597EFF069
:10487000FFE0F1BF411106C64922EF00E07BEF00E7
:10488000102C0100B24041018280011106CE02C607
:10489000EF00C0722A878547630CF70017C5010037
:1048A00013054594EFF09FDDB24793E727003EC61E
:1048B000EF0030212A878547630CF70017C50100F8
:1048C00013058594EFF09FDBB24793E747003EC6A0
:1048D000EF0090662A878547630CF70017C5010033
:1048E00013050595EFF09FD9B24793E787003EC6C1
:1048F000B2473E85F24005618280011106CE02C6B4
:10490000953F170700001307670481460546930586
:10491000400617C501001305E593EFE01F982AC66E
:10492000B24799CBEFD04FC2AA87014781463E8656
:1049300085453245EFE09F9C02C4EFD08FA08147B0
:104940003E85F24005618280797106D62AC697C7F6
:104950000100938767B49C431387470697C70100FC
:10496000938787B398C397C70100938727B39C4366
:104970001387470697C70100938747B298C397C725
:104980000100938767B198438567938777BB63D5A9
:10499000E70497C70100938727B09843FD77938773
:1049A00087443E9797C70100938707AF98C3F13DAF
:1049B0002ACEF24799EB97C70100938727AE984319
:1049C00089679387773263DBE700F2473E85EFF034
:1049D000DFC9EFD0EF9E21A0010011A00100B2506D
:1049E000456182807370043001A001008280411112
:1049F0002AC62EC47370043001A0411106C60146B8
:104A000091451545EFB03FD52A8797570300938707
:104A100067D398C3975703009387C7D29C4397C522
:104A200001009385E5833E85EFC0EFFB8148014897
:104A30008147094781461306004097C501009385C9
:104A40006583170500001305C503EFC01F89814862
:104A5000014897570300938727CF054781461306E0
:104A6000004097C501009385658117050000130577
:104A70008541EFC09F860100B240410182803971BB
:104A800006DE2AC602D0A5A882572947B317F70029
:104A90003ED6EFD06FAB2AD497570300938787CACF
:104AA0009C43780881463256BA853E85EFC00F9800
:104AB000AA8799C7975703009387C7C9054798C323
:104AC000EFD08FA82A87A257B307F7403ED21257DC
:104AD000B2576378F700975703009387A7C7054736
:104AE00098C3B257BD07125763F8E7009757030002
:104AF000938747C6054798C3825785073ED002571C
:104B00009147E3D3E7F802D015A89757030093879E
:104B100067C39C43181081460146BA853E85EFB0B5
:104B20003FE42A8785476308F70097570300938778
:104B300067C2054798C3825785073ED00257914701
:104B4000E3D5E7FC02D0A5A882572947B317F700A1
:104B50003ED6EFD06F9F2AD497570300938787BE26
:104B60009C43181081463256BA853E85EFB05FDF10
:104B7000AA8799C7975703009387C7BD054798C36E
:104B8000EFD08F9C2A87A257B307F7403ED2125727
:104B9000B2576378F700975703009387A7BB054781
:104BA00098C3B257BD07125763F8E7009757030041
:104BB000938747BA054798C3825785073ED0025767
:104BC0009147E3D3E7F8975703009387E7B823A00B
:104BD000070097570300938727B79C433E85EFC094
:104BE000DFDF21A05145EFC07FA2975703009387D5
:104BF000A7B6984393075005E316F7FE5145EFC05B
:104C0000FFA097570300938727B523A0070002D082
:104C1000C1A0975703009387E7B29C437808814669
:104C20000146BA853E85EFC06F802A8785476308B5
:104C3000F700975703009387E7B1054798C3975745
:104C40000300938727B09C43181081460146BA851C
:104C50003E85EFB0FFD02A8785476308F700975756
:104C60000300938727AF054798C39757030093879F
:104C7000A7AE9843930750056318F70097570300B2
:104C8000938747AD054798C3975703009387C7ABF2
:104C90009C4391453E85EFC0DFAD97570300938756
:104CA000A7AB9843930750056318F7009757030085
:104CB000938747AA054798C3975703009387C7A8C8
:104CC0009C4385453E85EFC0DFAA825785073ED0CD
:104CD00002579147E3DFE7F221A05145EFC01F9350
:104CE00097570300938747A7984393075005E31608
:104CF000F7FE5145EFC09F91975703009387C7A5D3
:104D000023A0070002D015A897570300938787A315
:104D10009C43780881460146BA853E85EFB01FF175
:104D20002A8785476308F70097570300938787A270
:104D3000054798C3825785073ED002579147E3D570
:104D4000E7FC97570300938727A09C433E85EFC05D
:104D5000DFC821A05145EFC07F8B97570300938791
:104D6000A79F984393075005E316F7FE5145EFC000
:104D7000FF89975703009387279E23A0070002D03F
:104D8000C1A0975703009387E79B9C431810814667
:104D90000146BA853E85EFB0BFBC2A8785476308C8
:104DA000F700975703009387E79A054798C39757EB
:104DB0000300938727999C43780881460146BA856A
:104DC0003E85EFB0BFE62A8785476308F70097570F
:104DD000030093872798054798C397570300938745
:104DE000A7979843930750056318F7009757030058
:104DF00093874796054798C3975703009387C794AF
:104E00009C4391453E85EFC0DF96975703009387FB
:104E1000A7949843930750056318F700975703002A
:104E200093874793054798C3975703009387C79184
:104E30009C4385453E85EFC0DF93825785073ED072
:104E400002579147E3DFE7F221A05145EFC00FFC85
:104E50009757030093874790984393075005E316AD
:104E6000F7FE5145EFC08FFA975703009387078EDF
:104E70009C4313871700975703009387278D98C388
:104E800011B1797106D62AC60145EFC0FFA2EFC065
:104E9000BFEB2ACE02CA975703009387E78B13070D
:104EA000500598C3975703009387C7899C435808B8
:104EB00081461306F00ABA853E85EFB07FAAAA871D
:104EC00099C7975703009387E788054798C3EFC0B2
:104ED000BFE72A87F247B307F7403ECC6247930704
:104EE000E00A63E8E700975703009387A786054722
:104EF00098C362479307E00B63F8E70097570300F6
:104F000093874785054798C3975703009387C784BE
:104F10001307500598C30145EFC01F9AEFC0DFE2A9
:104F20002ACE97570300938727831307500598C30A
:104F300097570300938707819C43580881461306BF
:104F4000F00ABA853E85EFB07FCEAA8799C79757FA
:104F5000030093872780054798C3EFC0FFDE2A87A9
:104F6000F247B307F7403ECC62479307E00A63E895
:104F7000E700974703009387E77D054798C362479B
:104F80009307E00B63F8E700974703009387877C5C
:104F9000054798C3974703009387077C130750057D
:104FA00098C3974703009387A77A9C4313871700FA
:104FB000974703009387C77998C3F9B5411185478F
:104FC0003EC6974703009387677898439747030047
:104FD0009387C7789C436313F70002C69747030083
:104FE00093870777984397470300938767779C4396
:104FF0006313F70002C6974703009387A77598438A
:1050000085476313F70002C69747030093874774E9
:105010009843974703009387A77498C39747030063
:105020009387C7729843974703009387277398C362
:10503000B2473E8541018280411106C69305800C2E
:105040001305800CEFB05F8D2A8797470300938785
:10505000A77198C397470300938707711307A00AA6
:10506000D8C3974703009387277023A4070081457F
:105070001305800CEFB05F8A2A8797470300938758
:10508000A76ED8C7974703009387076E23A807002A
:10509000974703009387476D23AA070097470300AC
:1050A0009387876C9C4397B501009385A51D3E852A
:1050B000EFC06F93974703009387076BDC4797B563
:1050C00001009385251D3E85EFC0EF9197470300B2
:1050D000938787699C4399E7974703009387C7683D
:1050E000DC47A9CB81480148814701479746030027
:1050F000938686671306004097B501009385851A4D
:10510000170500001305C515EFC02F9D8148014804
:1051100081470147974603009386C6651306004002
:1051200097B50100938585181705000013054513F1
:10513000EFC0AF9A0100B24041018280797106D67A
:105140002AC62EC48146014681453245EFB05F81B3
:105150002A8785476318F70097470300938787607E
:10516000054798C302CE15A88146014681453245C0
:10517000EFB0DFAB2A8785476308F7009747030046
:105180009387475E054798C3A2479C431387170040
:10519000A24798C3F24785073ECE72479307700C2B
:1051A000E3F4E7FC8146014681453245EFB01FA894
:1051B0002A8785476318F700974703009387875A24
:1051C000054798C30100B25045618280797106D6C7
:1051D0002AC62EC48146014681453245EFB01FA53F
:1051E0002A8785476318F7009747030093878757F7
:1051F000054798C302CE15A8814601468145324530
:10520000EFB00FF62A8785476308F700974703003A
:1052100093874755054798C3A2479C4313871700B8
:10522000A24798C3F24785073ECE72479307700C9A
:10523000E3F4E7FC8146014681453245EFB04FF289
:105240002A8785476318F70097470300938787519C
:10525000054798C30100B25045618280797106D636
:105260002AC6B2473ECEF247D8439307A00A631935
:10527000F700F2479843F247A107BE853A857D3D86
:10528000F2479C438146014681453E85EFB01F9A17
:105290002A8785476318F700974703009387874C51
:1052A000054798C3F2479843F247A107BE853A8560
:1052B000313FF2479843F247A107BE853A85BD3D8D
:1052C000D5B7411185473EC6974703009387874965
:1052D0009C4391C302C6974703009387E7489847CA
:1052E000974703009387C7499C436314F70002C69E
:1052F00019A89747030093872747984797470300C4
:105300009387074898C3974703009387E745D84B8F
:1053100097470300938707479C436314F70002C62F
:1053200019A89747030093872744D84B9747030052
:105330009387474598C3B2473E854101828041111A
:1053400006C61145EFB0EFC92A8797470300938738
:10535000A74398C397470300938707439C4397B598
:105360000100938525F53E85EFB0FFE797470300E1
:10537000938787419C43B5CB8148014897470300F9
:1053800093874742094781461306004097B50100BD
:10539000938545F3170500001305E505EFB0FFF30E
:1053A0008148014897470300938707400547814696
:1053B0001306004097B50100938545F117050000DD
:1053C00013056513EFB07FF181480148814701471C
:1053D00081461306004097B501009385A5EF170598
:1053E00000001305451EEFB05FEF0100B240410120
:1053F0008280797106D62AC6974703009387C738FB
:105400009C433E85EFB0CFC52A8785476318F700D8
:105410009747030093878737054798C302CE15A89F
:1054200097470300938747369C43A1453E85EFB0DD
:105430006FC82A8785476308F7009747030093875B
:10544000E734054798C35145EFC04F9CF2478507A5
:105450003ECE7247A547E3F5E7FC02CE0DA85145C5
:10546000EFC0CF9A97470300938707329C433E854E
:10547000EFB00FBF2A8785476308F70097470300FF
:105480009387C730054798C3F24785073ECE7247DA
:10549000A547E3F6E7FC974703009387E72E9C4375
:1054A0003E85EFB0EFBB2A8785476318F700974723
:1054B00003009387A72D054798C397470300938759
:1054C000A72D9C4313871700974703009387C72C8A
:1054D00098C3974703009387A72B054798C30145B7
:1054E000EFC08FBD974703009387872A23A007004B
:1054F00021B7011106CE2AC6974703009387C72814
:105500009C43F9553E85EFB0EFBA2A878547631370
:10551000F706974703009387A727984385476309B2
:10552000F7009747030093876726054798C389A824
:1055300097470300938747259C433E85EFB04FB2C2
:105540002A8785476308F700974703009387072456
:10555000054798C3974703009387C723054798C318
:105560000145EFC06FB5974703009387A72223A09B
:10557000070039A09747030093874721054798C341
:1055800097470300938787219C431387170097470A
:105590000300938767209C436308F7009747030045
:1055A0009387C71E054798C3974703009387071F34
:1055B0009C4313871700974703009387271E98C3C0
:1055C00025BF011106CE2AC6974703009387C71B44
:1055D0009C4381453E85EFB0EFAD2A878547E315B3
:1055E000F7FE974703009387E71B9C433E85EFC078
:1055F000AF872A878D476305F7007370043001A0D9
:10560000974703009387471A9C433E85EFC0CF8599
:105610002A878D476305F7007370043001A0974710
:1056200003009387271798438547631AF700974726
:1056300003009387E715984385476309F700974769
:1056400003009387A714054798C3F5A09747030065
:10565000938707159C431387170097470300938789
:10566000271498C397470300938707149C433E85EC
:10567000EFC0AFB6974703009387C7129C433E85A0
:10568000EFC0AFB5974703009387C710984385478E
:10569000630AF700974703009387870F984385476E
:1056A0006318F700974703009387470E054798C391
:1056B0000145EFC04F852A8789476305F70073705E
:1056C000043001A0974703009387C70D9C433E8594
:1056D000EFB09FF92A8789476305F700737004309C
:1056E00001A0974703009387270C9C433E85EFB0AA
:1056F000BFF72A8789476305F7007370043001A05C
:1057000097470300938747089C433E85EFB04F952A
:105710002A8785476308F7009747030093870707A1
:10572000054798C30145EFB01FFEAA87E38E07E83F
:105730007370043001A049BD41119747030093875E
:10574000E706984397470300938707059C4363192F
:10575000F7009747030093876703054798C319A885
:10576000974703009387470398439747030093871E
:10577000E70398C3974703009387870398439747A6
:1057800003009387A7019C436319F7009747030021
:105790009387C7FF054798C319A8974703009387C6
:1057A000E7FF9843974703009387870098C397477D
:1057B000030093872700984397470300938747FE8A
:1057C0009C436319F70097470300938727FC05471D
:1057D00098C319A897470300938787FC9843974776
:1057E0000300938727FD98C397470300938707FA21
:1057F000984385476314F70002C619A085473EC643
:10580000B2473E8541018280B305B500930705008C
:105810006386B70003C70700631607003385A740F8
:1058200067800000938717006FF09FFE130101FD52
:1058300023229102232A51012326110223248102CB
:1058400023202103232E3101232C41012328610130
:105850002326710123248101232291012320A10108
:10586000930A050093840500639E0638130406001E
:105870009309050017B90100130949A663F8C51279
:10588000B7070100138B05006378F6101307F00FBC
:105890003337C70013173700B357E6003309F90051
:1058A000834609003387E60093060002B386E6408C
:1058B000638C0600B394D40033D7EA003314D600C7
:1058C000336B9700B399DA00935A040193850A0069
:1058D00013050B00EF00902A1309050093850A00B9
:1058E000931B040113050B00EF00D02493DB0B0185
:1058F000930405009305050013850B00EF00D020ED
:105900001319090193D70901B367F900138A040039
:1059100063FEA700B3878700138AF4FF63E887005C
:1059200063F6A700138AE4FFB3878700B384A74018
:1059300093850A0013850400EF0050241309050025
:1059400093850A0013850400EF00D01E9399090186
:1059500093040500930505001319090113850B0035
:1059600093D90901EF00501AB36939011386040075
:1059700063FCA900B30934011386F4FF63E68900D0
:1059800063F4A9001386E4FF13140A013364C4000E
:10599000130A00006F000013B7070001130700018E
:1059A000E36CF6EE130780016FF01FEF138A060019
:1059B000631A06009305000013051000EF0090170E
:1059C00013040500B7070100637EF4129307F00F7C
:1059D00063F48700130A8000B35744013309F900C8
:1059E000034709009306000233074701B386E640E8
:1059F00063940612B3848440130A1000135B0401FD
:105A000093050B0013850400EF00501713090500E0
:105A100093050B0013850400931B0401EF00901104
:105A200093DB0B01930405009305050013850B0020
:105A3000EF00900D1319090193D70901B367F9001D
:105A4000938A040063FEA700B3878700938AF4FF5C
:105A500063E8870063F6A700938AE4FFB3878700B3
:105A6000B384A74093050B0013850400EF001011C9
:105A70001309050093050B0013850400EF00900B3C
:105A80009399090193040500930505001319090171
:105A900013850B0093D90901EF001007B369390191
:105AA0001386040063FCA900B30934011386F4FFD4
:105AB00063E6890063F4A9001386E4FF13940A01E6
:105AC0003364C4001305040093050A008320C10257
:105AD0000324810283244102032901028329C10195
:105AE000032A8101832A4101032B0101832BC10079
:105AF000032C8100832C4100032D010013010103BD
:105B000067800000B7070001130A0001E366F4ECA8
:105B1000130A80016FF05FEC3314D40033DAE40031
:105B2000B399DA0033D7EA00935A0401B394D4004E
:105B300093850A0013050A00336B9700EF001004E9
:105B40001309050093850A0013050A00931B04013D
:105B5000EF00407E93DB0B019304050093050500E5
:105B600013850B00EF00407A1319090113570B013D
:105B70003367E900138A0400637EA70033078700B8
:105B8000138AF4FF636887006376A700138AE4FF33
:105B900033078700B304A74093850A0013850400E8
:105BA000EF00C07D1309050093850A0013850400EA
:105BB000EF004078930405009305050013850B0062
:105BC000EF00807413170B01135707011319090114
:105BD000B367E9001387040063FEA700B38787005B
:105BE0001387F4FF63E8870063F6A7001387E4FFD9
:105BF000B3878700131A0A01B384A740336AEA0007
:105C00006FF0DFDF63ECD51EB707010063F4F60425
:105C10001307F00FB335D7009395350033D7B6008F
:105C200097A701009387876BB387E70003C7070037
:105C3000130A00023307B700330AEA4063160A0268
:105C400013041000E3E096E833B6CA0013441600CC
:105C50006FF05FE7B707000193050001E3E0F6FC92
:105C6000930580016FF09FFBB35CE600B39646019D
:105C7000B3ECDC0033D4E40093DB0C01B3974401B4
:105C800033D7EA0093850B0013050400336BF7004C
:105C9000B3194601EF00806E1309050093850B00D0
:105CA00013050400139C0C01EF00C068135C0C0189
:105CB000930405009305050013050C00EF00C06474
:105CC0001319090113570B013367E900138404000A
:105CD000637EA700330797011384F4FF636897017D
:105CE0006376A7001384E4FF33079701B304A7404A
:105CF00093850B0013850400EF004068130905002D
:105D000093850B0013850400EF00C0629304050027
:105D10009305050013050C00EF00005F93170B01BE
:105D20001319090193D70701B367F900138604001B
:105D300063FEA700B38797011386F4FF63E897011A
:105D400063F6A7001386E4FFB387970113140401D9
:105D5000B70B01003364C4001389FBFF337D2401BA
:105D600033F92901B384A7409305090013050D00F9
:105D7000EF008059935C040193050900130B0500A3
:105D800013850C00EF00405893D90901130C05004E
:105D90009385090013850C00EF00005713090500D7
:105DA0009385090013050D00EF00005633058501AA
:105DB00093570B013385A70063748501330979017B
:105DC00093570501B387270163E6F402E392F4BC1D
:105DD000B70701009387F7FF3375F5001315050129
:105DE000337BFB0033964A0133056501130A00003B
:105DF000E37AA6CC1304F4FF6FF09FB9130A0000F6
:105E0000130400006FF01FCC130101FB2324810455
:105E100023229104232E31032322910323261104EC
:105E200023202105232C4103232A51032328610326
:105E300023267103232481032320A103232EB101F0
:105E4000930C050093890500130405009384050055
:105E5000639E062613090600138A060097AA01000E
:105E6000938ACA4763F4C514B70701006376F61234
:105E70009307F00F63F4C700130A8000B35746017D
:105E8000B38AFA0003C70A0013050002330747016B
:105E9000330AE540630C0A00B395490133D7EC009F
:105EA00033194601B364B70033944C01935A090186
:105EB00093850A0013850400EF00404C9309050008
:105EC00093850A00131B090113850400EF00804627
:105ED000135B0B019305050013050B00EF00C04297
:105EE0009399090193570401B3E7F90063FAA700F6
:105EF000B387270163E6270163F4A700B38727016F
:105F0000B384A74093850A0013850400EF0000477F
:105F10009309050093850A0013850400EF00804172
:105F200013140401930505009399090113050B004F
:105F300013540401EF00403D33E48900637AA40068
:105F400033042401636624016374A4003304240130
:105F50003304A44033554401930500008320C10459
:105F60000324810483244104032901048329C103F8
:105F7000032A8103832A4103032B0103832BC102DC
:105F8000032C8102832C4102032D0102832DC101C8
:105F90001301010567800000B7070001130A000123
:105FA000E36EF6EC130A80016FF05FED631A0600F2
:105FB0009305000013051000EF00C037130905001A
:105FC000B7070100637AF90E9307F00F63F4270116
:105FD000130A8000B3574901B38AFA0003C70A00C5
:105FE00013050002B384294133074701330AE54012
:105FF000E30E0AEA33194901B3DAE900B39549011E
:1060000033D7EC0093540901336BB70013850A00B2
:1060100093850400EF008036930905009385040002
:10602000931B090113850A00EF00C03093DB0B01BD
:106030009305050013850B00EF00002D93990901CE
:1060400093570B01B3E7F90033944C0163FAA700AF
:10605000B387270163E6270163F4A700B38727010D
:10606000B38AA7409385040013850A00EF0000312E
:10607000930905009385040013850A00EF00802B27
:106080009305050013850B00EF00002893150B0105
:106090009399090193D50501B3E5B90063FAA50009
:1060A000B385250163E6250163F4A500B3852501C9
:1060B000B384A5406FF09FDFB7070001130A00010A
:1060C000E36AF9F0130A80016FF0DFF0E3E8D5E846
:1060D000B707010063FCF604930BF00F33B5DB0048
:1060E0001315350033D7A60097A701009387071F24
:1060F000B387E70083CB070093050002B38BAB00A7
:10610000338B7541631E0B0263E4360163EACC00F6
:106110003384CC40B386D94033B58C00B384A640D9
:1061200013050400938504006FF05FE3B7070001D7
:1061300013050001E3E8F6FA130580016FF09FFAFA
:10614000B3966601335D7601336DDD0033D479019A
:10615000B395690133DC7C0193540D01336CBC00B1
:106160001305040093850400B31A6601EF000021B3
:10617000130A0500938504001305040033996C018C
:10618000931C0D01EF00001B93DC0C0113040500B0
:106190009305050013850C00EF000017131A0A0180
:1061A00013570C013367EA00130A0400637EA7004B
:1061B0003307A701130AF4FF6368A7016376A700FA
:1061C000130AE4FF3307A701B309A740938504002E
:1061D00013850900EF00801A93850400130405005D
:1061E00013850900EF0000159305050093040500D1
:1061F00013850C00EF00401193150C0113140401DA
:1062000093D50501B365B4001387040063FEA500B0
:10621000B385A5011387F4FF63E8A50163F6A50024
:106220001387E4FFB385A501131A0A01B70C010017
:10623000336AEA001384FCFFB3778A0033F48A00E0
:10624000B384A54013850700930504002326F100BD
:10625000135A0A01EF00400B93090500930504004F
:1062600013050A00EF00400A13DC0A01930D050034
:1062700093050C0013050A00EF0000098327C100F5
:10628000130A050093050C0013850700EF00C007F3
:106290003305B50113D709013307A7006374B701AC
:1062A000330A9A01B70701009387F7FF9355070157
:1062B0003377F70013170701B3F7F900B3854501EA
:1062C000B307F70063E6B400639EB400637CF90093
:1062D00033865741B3B7C700B385A541B385F540B1
:1062E00093070600B307F9403339F900B385B4408A
:1062F000B385254133947501B3D767013365F40045
:10630000B3D565016FF09FC51306050013050000A6
:1063100093F61500638406003305C50093D5150078
:1063200013161600E39605FE67800000634005061D
:1063300063C6050613860500930505001305F0FFE7
:10634000630C060293061000637AB6006358C0001F
:106350001316160093961600E36AB6FE13050000A6
:1063600063E6C500B385C5403365D50093D61600F6
:1063700013561600E39606FE678000009382000025
:10638000EFF05FFB13850500678002003305A04036
:1063900063D80500B305B0406FF0DFF9B305B04036
:1063A00093820000EFF01FF93305A04067800200E0
:1063B0009382000063CA0500634C0500EFF09FF76D
:1063C0001385050067800200B305B040E35805FE61
:1063D0003305A040EFF01FF63305B04067800200A0
:02000004800278
:1000000049444C4500000000482FFEFF102FFEFF22
:100010001E2FFEFF2C2FFEFF342FFEFF5830FEFF59
:100020002030FEFF2E30FEFF3C30FEFF4430FEFF4E
:10003000546D722053766300DC35FEFFDC35FEFF25
:10004000DC35FEFF5A36FEFF2A36FEFF5036FEFF35
:10005000DC35FEFFDC35FEFF5A36FEFF2A36FEFF9A
:10006000546D725100000000286E756C6C29000000
:10007000DE43FEFFDC45FEFFD245FEFFDC45FEFF12
:10008000DC45FEFFDC45FEFFDC45FEFF5C44FEFF79
:10009000DC45FEFFDC45FEFF1444FEFF6A44FEFF24
:1000A000DC45FEFF1E44FEFF2844FEFF2844FEFF01
:1000B0002844FEFF2844FEFF2844FEFF2844FEFF9C
:1000C0002844FEFF2844FEFF2844FEFFDC45FEFFD7
:1000D000DC45FEFFDC45FEFFDC45FEFFDC45FEFFA8
:1000E000DC45FEFFDC45FEFFDC45FEFFDC45FEFF98
:1000F000DC45FEFFDC45FEFFDC45FEFFDC45FEFF88
:10010000DC45FEFFDC45FEFFDC45FEFFDC45FEFF77
:10011000DC45FEFFDC45FEFFDC45FEFFDC45FEFF67
:10012000DC45FEFFDC45FEFFDC45FEFFDC45FEFF57
:10013000DC45FEFFDC45FEFFDC45FEFFDC45FEFF47
:10014000DC45FEFFDC45FEFFDC45FEFFDC45FEFF37
:10015000DC45FEFFDC45FEFFDC45FEFFDC45FEFF27
:10016000DC45FEFFDC45FEFFDC45FEFFDC45FEFF17
:100170008E44FEFF3A45FEFFDC45FEFFDC45FEFFF8
:10018000DC45FEFFDC45FEFFDC45FEFFDC45FEFFF7
:10019000DC45FEFF8644FEFFDC45FEFFDC45FEFF3E
:1001A0008E45FEFF9445FEFFDC45FEFFDC45FEFF6D
:1001B000A244FEFFDC45FEFF8845FEFFDC45FEFF56
:1001C000DC45FEFFAC45FEFF6D69616F750A0000FE
:1001D0006D69616F75320A0068756E6772790A0021
:1001E0004572726F7220696E20626C6F636B20744F
:1001F000696D652074657374207461736B73200D71
:100200000A0000004572726F7220696E20636F757C
:100210006E74696E672073656D6170686F726520BA
:100220007461736B73200D0A000000004572726FD9
:100230007220696E20726563757273697665206DD0
:1002400075746578207461736B73200D0A0000006B
:10025000436865636B54696D65720000426C6F633F
:100260006B5F54696D655F517565756500000000D1
:100270004254657374310000425465737432000057
:10028000436F756E74696E675F53656D5F31000013
:10029000436F756E74696E675F53656D5F32000002
:1002A000434E543100000000434E54320000000021
:1002B0005265637572736976655F4D757465780014
:1002C0005265633100000000526563320000000097
:1002D00052656333000000000001020203030303C0
:1002E00004040404040404040505050505050505C6
:1002F00005050505050505050606060606060606A6
:10030000060606060606060606060606060606068D
:100310000606060606060606070707070707070775
:10032000070707070707070707070707070707075D
:10033000070707070707070707070707070707074D
:10034000070707070707070707070707070707073D
:100350000707070707070707080808080808080825
:10036000080808080808080808080808080808080D
:1003700008080808080808080808080808080808FD
:1003800008080808080808080808080808080808ED
:1003900008080808080808080808080808080808DD
:1003A00008080808080808080808080808080808CD
:1003B00008080808080808080808080808080808BD
:1003C00008080808080808080808080808080808AD
:0803D0000808080808080808E5
:1003D8001000000000000000017A5200017C0101B9
:1003E8001B0D02004C000000180000003854FEFFEE
:1003F800DC05000000440E307089039507810188F0
:100408000292049305940696089709980A990B9AFC
:100418000C0370020AC144C844C944D244D344D42A
:1004280044D544D644D744D844D944DA440E004489
:100438000B0000005000000068000000C459FEFFD7
:100448000005000000440E50748802890393059942
:100458000B810192049406950796089709980A9AC1
:100468000C9B0D0320010AC144C844C944D244D39B
:1004780044D444D544D644D744D844D944DA44DB98
:08048800440E00440B000000CB
:10049C00AAAAAAAA08000000FC8F01000400000010
:040000058000004037
:00000001FF
